:1000000000308A0080280000FF00030E8301A10059
:100010007F08A0000A08A8008A01A00E0408A20018
:100020007708A3007808A4007908A5007A08A6003C
:100030007B08A700831383128B1E20280B193328FB
:10004000220884002308F7002408F8002508F90096
:100050002608FA002708FB0028088A00210E8300E2
:10006000FF0E7F0E0900B501290B4C28B43081002A
:100070002D302B0784008008031940282C088804A1
:100080000310AC0DAC08031D47280130AC00013053
:10009000A907AA01B50069282908023C031D5928AF
:1000A0002D302B0784000008FF3C81000330A9009D
:1000B00069282908033C031D692888012D302B0776
:1000C0008400000881000130AB070730AB05013028
:1000D000A9000B110B118A11202837308400000869
:1000E00003197F280630F800F701F70B7528F80B85
:1000F00074287B30F700F70B7B28800B72280034C4
:1001000084011F308305063083169F000A30990052
:1001100026309800903083129800A901AA01AB0103
:100120000130AC00AD01AE01AF01B001B101B201CF
:10013000B301B401B501B601B608031DA4288316A6
:10014000061083120614A8288316061183120615BA
:100150000130B600B608031DB228831606108312BC
:100160000610B62883160611831206110430B60055
:10017000FA30B7006D20B60BB828B601B608031DDB
:10018000C6288316061083120610CA288316061185
:10019000831206110130B600B608031DD428831659
:1001A000061083120614D82883160611831206152A
:1001B0000430B600FA30B7006D20B60BDA289B2861
:0201C0006300DA
:02400E00FA3F77
:00000001FF
